 EditCase

 Timestamp is 5685d13e (Fri Jan 01 04:07:10 2016)

 Preferred load address is 10000000

 Start         Length     Name                   Class
 0001:00000000 000000f8H .idata$5                CODE
 0001:000000f8 00000004H .CRT$XCA                CODE
 0001:000000fc 00000004H .CRT$XCZ                CODE
 0001:00000100 00000004H .CRT$XIA                CODE
 0001:00000104 0000000cH .CRT$XIC                CODE
 0001:00000110 00000004H .CRT$XIZ                CODE
 0001:00000114 00000004H .CRT$XPA                CODE
 0001:00000118 00000004H .CRT$XPZ                CODE
 0001:0000011c 00000004H .CRT$XTA                CODE
 0001:00000120 00000004H .CRT$XTZ                CODE
 0001:00000128 00001888H .rdata                  CODE
 0001:000019b0 0000000cH .rdata$sxdata           CODE
 0001:000019bc 00000004H .rtc$IAA                CODE
 0001:000019c0 00000004H .rtc$IZZ                CODE
 0001:000019c4 00000004H .rtc$TAA                CODE
 0001:000019c8 00000004H .rtc$TZZ                CODE
 0001:000019d0 000051b2H .text                   CODE
 0001:00006b88 000001acH .xdata$x                CODE
 0001:00006d34 00000014H .idata$2                CODE
 0001:00006d48 00000014H .idata$3                CODE
 0001:00006d5c 000000f8H .idata$4                CODE
 0001:00006e54 00000452H .idata$6                CODE
 0001:000072b0 000000a4H .edata                  CODE
 0002:00000000 00000b40H .data                   DATA
 0002:00000b40 00000f00H .bss                    DATA
 0003:00000000 00000058H .rsrc$01                DATA
 0003:00000060 00000388H .rsrc$02                DATA

  Address         Publics by Value              Rva+Base       Lib:Object

 0000:00000000       __except_list              00000000     <absolute>
 0000:00000003       ___safe_se_handler_count   00000003     <absolute>
 0000:00000000       ___ImageBase               10000000     <linker-defined>
 0001:00000000       __imp__lstrcatW@8          10001000     kernel32:KERNEL32.dll
 0001:00000004       __imp__lstrcpyW@8          10001004     kernel32:KERNEL32.dll
 0001:00000008       __imp__lstrlenW@4          10001008     kernel32:KERNEL32.dll
 0001:0000000c       __imp__lstrcmpW@8          1000100c     kernel32:KERNEL32.dll
 0001:00000010       __imp__lstrcpynW@12        10001010     kernel32:KERNEL32.dll
 0001:00000014       __imp__lstrcmpiW@8         10001014     kernel32:KERNEL32.dll
 0001:00000018       __imp__HeapAlloc@12        10001018     kernel32:KERNEL32.dll
 0001:0000001c       __imp__GetLastError@0      1000101c     kernel32:KERNEL32.dll
 0001:00000020       __imp__HeapFree@12         10001020     kernel32:KERNEL32.dll
 0001:00000024       __imp__GetCurrentThreadId@0 10001024     kernel32:KERNEL32.dll
 0001:00000028       __imp__DecodePointer@4     10001028     kernel32:KERNEL32.dll
 0001:0000002c       __imp__GetCommandLineA@0   1000102c     kernel32:KERNEL32.dll
 0001:00000030       __imp__IsProcessorFeaturePresent@4 10001030     kernel32:KERNEL32.dll
 0001:00000034       __imp__GetProcAddress@8    10001034     kernel32:KERNEL32.dll
 0001:00000038       __imp__GetModuleHandleW@4  10001038     kernel32:KERNEL32.dll
 0001:0000003c       __imp__ExitProcess@4       1000103c     kernel32:KERNEL32.dll
 0001:00000040       __imp__WriteFile@20        10001040     kernel32:KERNEL32.dll
 0001:00000044       __imp__GetStdHandle@4      10001044     kernel32:KERNEL32.dll
 0001:00000048       __imp__GetModuleFileNameW@12 10001048     kernel32:KERNEL32.dll
 0001:0000004c       __imp__HeapCreate@12       1000104c     kernel32:KERNEL32.dll
 0001:00000050       __imp__HeapDestroy@4       10001050     kernel32:KERNEL32.dll
 0001:00000054       __imp__EncodePointer@4     10001054     kernel32:KERNEL32.dll
 0001:00000058       __imp__TlsAlloc@0          10001058     kernel32:KERNEL32.dll
 0001:0000005c       __imp__TlsGetValue@4       1000105c     kernel32:KERNEL32.dll
 0001:00000060       __imp__TlsSetValue@8       10001060     kernel32:KERNEL32.dll
 0001:00000064       __imp__TlsFree@4           10001064     kernel32:KERNEL32.dll
 0001:00000068       __imp__InterlockedIncrement@4 10001068     kernel32:KERNEL32.dll
 0001:0000006c       __imp__SetLastError@4      1000106c     kernel32:KERNEL32.dll
 0001:00000070       __imp__InterlockedDecrement@4 10001070     kernel32:KERNEL32.dll
 0001:00000074       __imp__Sleep@4             10001074     kernel32:KERNEL32.dll
 0001:00000078       __imp__SetHandleCount@4    10001078     kernel32:KERNEL32.dll
 0001:0000007c       __imp__InitializeCriticalSectionAndSpinCount@8 1000107c     kernel32:KERNEL32.dll
 0001:00000080       __imp__GetFileType@4       10001080     kernel32:KERNEL32.dll
 0001:00000084       __imp__GetStartupInfoW@4   10001084     kernel32:KERNEL32.dll
 0001:00000088       __imp__DeleteCriticalSection@4 10001088     kernel32:KERNEL32.dll
 0001:0000008c       __imp__GetModuleFileNameA@12 1000108c     kernel32:KERNEL32.dll
 0001:00000090       __imp__FreeEnvironmentStringsW@4 10001090     kernel32:KERNEL32.dll
 0001:00000094       __imp__WideCharToMultiByte@32 10001094     kernel32:KERNEL32.dll
 0001:00000098       __imp__GetEnvironmentStringsW@0 10001098     kernel32:KERNEL32.dll
 0001:0000009c       __imp__QueryPerformanceCounter@4 1000109c     kernel32:KERNEL32.dll
 0001:000000a0       __imp__GetTickCount@0      100010a0     kernel32:KERNEL32.dll
 0001:000000a4       __imp__GetCurrentProcessId@0 100010a4     kernel32:KERNEL32.dll
 0001:000000a8       __imp__GetSystemTimeAsFileTime@4 100010a8     kernel32:KERNEL32.dll
 0001:000000ac       __imp__LeaveCriticalSection@4 100010ac     kernel32:KERNEL32.dll
 0001:000000b0       __imp__EnterCriticalSection@4 100010b0     kernel32:KERNEL32.dll
 0001:000000b4       __imp__LoadLibraryW@4      100010b4     kernel32:KERNEL32.dll
 0001:000000b8       __imp__UnhandledExceptionFilter@4 100010b8     kernel32:KERNEL32.dll
 0001:000000bc       __imp__SetUnhandledExceptionFilter@4 100010bc     kernel32:KERNEL32.dll
 0001:000000c0       __imp__IsDebuggerPresent@0 100010c0     kernel32:KERNEL32.dll
 0001:000000c4       __imp__TerminateProcess@8  100010c4     kernel32:KERNEL32.dll
 0001:000000c8       __imp__GetCurrentProcess@0 100010c8     kernel32:KERNEL32.dll
 0001:000000cc       __imp__GetCPInfo@8         100010cc     kernel32:KERNEL32.dll
 0001:000000d0       __imp__GetACP@0            100010d0     kernel32:KERNEL32.dll
 0001:000000d4       __imp__GetOEMCP@0          100010d4     kernel32:KERNEL32.dll
 0001:000000d8       __imp__IsValidCodePage@4   100010d8     kernel32:KERNEL32.dll
 0001:000000dc       __imp__HeapReAlloc@16      100010dc     kernel32:KERNEL32.dll
 0001:000000e0       __imp__RtlUnwind@16        100010e0     kernel32:KERNEL32.dll
 0001:000000e4       __imp__HeapSize@12         100010e4     kernel32:KERNEL32.dll
 0001:000000e8       __imp__LCMapStringW@24     100010e8     kernel32:KERNEL32.dll
 0001:000000ec       __imp__MultiByteToWideChar@24 100010ec     kernel32:KERNEL32.dll
 0001:000000f0       __imp__GetStringTypeW@16   100010f0     kernel32:KERNEL32.dll
 0001:000000f4       \177KERNEL32_NULL_THUNK_DATA 100010f4     kernel32:KERNEL32.dll
 0001:000000f8       ___xc_a                    100010f8     LIBCMT:crt0init.obj
 0001:000000fc       ___xc_z                    100010fc     LIBCMT:crt0init.obj
 0001:00000100       ___xi_a                    10001100     LIBCMT:crt0init.obj
 0001:00000110       ___xi_z                    10001110     LIBCMT:crt0init.obj
 0001:00000114       ___xp_a                    10001114     LIBCMT:crt0init.obj
 0001:00000118       ___xp_z                    10001118     LIBCMT:crt0init.obj
 0001:0000011c       ___xt_a                    1000111c     LIBCMT:crt0init.obj
 0001:00000120       ___xt_z                    10001120     LIBCMT:crt0init.obj
 0001:00000138       _MainGuid                  10001138     EditCase.obj
 0001:00000148       _MenuGuid                  10001148     EditCase.obj
 0001:00000158       ??_C@_1DE@BGKMIKPD@?$AAE?$AAu?$AAg?$AAe?$AAn?$AAe?$AA?5?$AAR?$AAo?$AAs?$AAh?$AAa?$AAl?$AA?5?$AA?$CG?$AA?5?$AAF?$AAa?$AAr?$AA?5?$AAG?$AAr?$AAo?$AAu?$AAp?$AA?$AA@ 10001158     EditCase.obj
 0001:00000190       ??_C@_1EK@IFCLLMMP@?$AAT?$AAe?$AAx?$AAt?$AA?5?$AAc?$AAa?$AAs?$AAe?$AA?5?$AAc?$AAo?$AAn?$AAv?$AAe?$AAr?$AAs?$AAi?$AAo?$AAn?$AA?5?$AAf?$AAo?$AAr?$AA?5?$AAF?$AAa?$AAr?$AA?5?$AAM?$AAa?$AAn@ 10001190     EditCase.obj
 0001:000001dc       ??_C@_1BC@MGKGEOAP@?$AAE?$AAd?$AAi?$AAt?$AAC?$AAa?$AAs?$AAe?$AA?$AA@ 100011dc     EditCase.obj
 0001:000001f0       ??_C@_19DHONEMF@?$AA?5?$AA?6?$AA?$AN?$AA?7?$AA?$AA@ 100011f0     EditCase.obj
 0001:000001fc       ??_C@_1BA@CAKIGJMA@?$AAW?$AAo?$AAr?$AAd?$AAD?$AAi?$AAv?$AA?$AA@ 100011fc     EditCase.obj
 0001:0000020c       ??_C@_13GMDMCADD@?$AA?$CD?$AA?$AA@ 1000120c     EditCase.obj
 0001:00000210       ??_C@_1BG@DENGNAGA@?$AAA?$AAd?$AAd?$AAW?$AAo?$AAr?$AAd?$AAD?$AAi?$AAv?$AA?$AA@ 10001210     EditCase.obj
 0001:00000228       ??_C@_1BC@ENICKDH@?$AAC?$AAo?$AAn?$AAt?$AAe?$AAn?$AAt?$AAs?$AA?$AA@ 10001228     EditCase.obj
 0001:0000023c       ??_C@_1M@LPIADJOF@?$AAL?$AAO?$AAW?$AAE?$AAR?$AA?$AA@ 1000123c     EditCase.obj
 0001:00000248       ??_C@_1M@NMMEOLKN@?$AAT?$AAI?$AAT?$AAL?$AAE?$AA?$AA@ 10001248     EditCase.obj
 0001:00000254       ??_C@_1M@PCFBDNPE@?$AAU?$AAP?$AAP?$AAE?$AAR?$AA?$AA@ 10001254     EditCase.obj
 0001:00000260       ??_C@_1O@NJHKFPAK@?$AAT?$AAO?$AAG?$AAG?$AAL?$AAE?$AA?$AA@ 10001260     EditCase.obj
 0001:00000270       ??_C@_1O@BIAHPDPJ@?$AAC?$AAY?$AAC?$AAL?$AAI?$AAC?$AA?$AA@ 10001270     EditCase.obj
 0001:00000280       __pDefaultRawDllMain       10001280     LIBCMT:dllcrt0.obj
 0001:00000280       __pRawDllMain              10001280     LIBCMT:dllcrt0.obj
 0001:00000284       ??_C@_0P@MIGLKIOC@CorExitProcess?$AA@ 10001284     LIBCMT:crt0dat.obj
 0001:00000294       ??_C@_1BI@BGOHAHKC@?$AAm?$AAs?$AAc?$AAo?$AAr?$AAe?$AAe?$AA?4?$AAd?$AAl?$AAl?$AA?$AA@ 10001294     LIBCMT:crt0dat.obj
 0001:000002ac       ??_C@_1BO@BKOMIGKJ@?$AAr?$AAu?$AAn?$AAt?$AAi?$AAm?$AAe?$AA?5?$AAe?$AAr?$AAr?$AAo?$AAr?$AA?5?$AA?$AA@ 100012ac     LIBCMT:crt0msg.obj
 0001:000002cc       ??_C@_15JNBOKNOG@?$AA?$AN?$AA?6?$AA?$AA@ 100012cc     LIBCMT:crt0msg.obj
 0001:000002d4       ??_C@_1BM@JBBEPPHI@?$AAT?$AAL?$AAO?$AAS?$AAS?$AA?5?$AAe?$AAr?$AAr?$AAo?$AAr?$AA?$AN?$AA?6?$AA?$AA@ 100012d4     LIBCMT:crt0msg.obj
 0001:000002f0       ??_C@_1BK@KMOMNAAI@?$AAS?$AAI?$AAN?$AAG?$AA?5?$AAe?$AAr?$AAr?$AAo?$AAr?$AA?$AN?$AA?6?$AA?$AA@ 100012f0     LIBCMT:crt0msg.obj
 0001:0000030c       ??_C@_1BO@BFCDCGC@?$AAD?$AAO?$AAM?$AAA?$AAI?$AAN?$AA?5?$AAe?$AAr?$AAr?$AAo?$AAr?$AA?$AN?$AA?6?$AA?$AA@ 1000130c     LIBCMT:crt0msg.obj
 0001:00000330       ??_C@_1BOO@KGEDBGAJ@?$AAR?$AA6?$AA0?$AA3?$AA3?$AA?$AN?$AA?6?$AA?9?$AA?5?$AAA?$AAt?$AAt?$AAe?$AAm?$AAp?$AAt?$AA?5?$AAt?$AAo?$AA?5?$AAu?$AAs?$AAe?$AA?5?$AAM?$AAS?$AAI?$AAL?$AA?5?$AAc?$AAo?$AAd@ 10001330     LIBCMT:crt0msg.obj
 0001:00000520       ??_C@_1GG@GOPILAJP@?$AAR?$AA6?$AA0?$AA3?$AA2?$AA?$AN?$AA?6?$AA?9?$AA?5?$AAn?$AAo?$AAt?$AA?5?$AAe?$AAn?$AAo?$AAu?$AAg?$AAh?$AA?5?$AAs?$AAp?$AAa?$AAc?$AAe?$AA?5?$AAf?$AAo?$AAr?$AA?5?$AAl?$AAo@ 10001520     LIBCMT:crt0msg.obj
 0001:00000588       ??_C@_1MG@ENCOOIDF@?$AAR?$AA6?$AA0?$AA3?$AA1?$AA?$AN?$AA?6?$AA?9?$AA?5?$AAA?$AAt?$AAt?$AAe?$AAm?$AAp?$AAt?$AA?5?$AAt?$AAo?$AA?5?$AAi?$AAn?$AAi?$AAt?$AAi?$AAa?$AAl?$AAi?$AAz?$AAe?$AA?5?$AAt@ 10001588     LIBCMT:crt0msg.obj
 0001:00000650       ??_C@_1DO@BMFCDCD@?$AAR?$AA6?$AA0?$AA3?$AA0?$AA?$AN?$AA?6?$AA?9?$AA?5?$AAC?$AAR?$AAT?$AA?5?$AAn?$AAo?$AAt?$AA?5?$AAi?$AAn?$AAi?$AAt?$AAi?$AAa?$AAl?$AAi?$AAz?$AAe?$AAd?$AA?$AN?$AA?6?$AA?$AA@ 10001650     LIBCMT:crt0msg.obj
 0001:00000690       ??_C@_1EK@HHFLMAOL@?$AAR?$AA6?$AA0?$AA2?$AA8?$AA?$AN?$AA?6?$AA?9?$AA?5?$AAu?$AAn?$AAa?$AAb?$AAl?$AAe?$AA?5?$AAt?$AAo?$AA?5?$AAi?$AAn?$AAi?$AAt?$AAi?$AAa?$AAl?$AAi?$AAz?$AAe?$AA?5?$AAh?$AAe@ 10001690     LIBCMT:crt0msg.obj
 0001:000006e0       ??_C@_1GK@MFGOKLAG@?$AAR?$AA6?$AA0?$AA2?$AA7?$AA?$AN?$AA?6?$AA?9?$AA?5?$AAn?$AAo?$AAt?$AA?5?$AAe?$AAn?$AAo?$AAu?$AAg?$AAh?$AA?5?$AAs?$AAp?$AAa?$AAc?$AAe?$AA?5?$AAf?$AAo?$AAr?$AA?5?$AAl?$AAo@ 100016e0     LIBCMT:crt0msg.obj
 0001:00000750       ??_C@_1GK@MCAAGJMO@?$AAR?$AA6?$AA0?$AA2?$AA6?$AA?$AN?$AA?6?$AA?9?$AA?5?$AAn?$AAo?$AAt?$AA?5?$AAe?$AAn?$AAo?$AAu?$AAg?$AAh?$AA?5?$AAs?$AAp?$AAa?$AAc?$AAe?$AA?5?$AAf?$AAo?$AAr?$AA?5?$AAs?$AAt@ 10001750     LIBCMT:crt0msg.obj
 0001:000007c0       ??_C@_1EM@MAADIHMB@?$AAR?$AA6?$AA0?$AA2?$AA5?$AA?$AN?$AA?6?$AA?9?$AA?5?$AAp?$AAu?$AAr?$AAe?$AA?5?$AAv?$AAi?$AAr?$AAt?$AAu?$AAa?$AAl?$AA?5?$AAf?$AAu?$AAn?$AAc?$AAt?$AAi?$AAo?$AAn?$AA?5?$AAc@ 100017c0     LIBCMT:crt0msg.obj
 0001:00000810       ??_C@_1GK@FHCKBEFA@?$AAR?$AA6?$AA0?$AA2?$AA4?$AA?$AN?$AA?6?$AA?9?$AA?5?$AAn?$AAo?$AAt?$AA?5?$AAe?$AAn?$AAo?$AAu?$AAg?$AAh?$AA?5?$AAs?$AAp?$AAa?$AAc?$AAe?$AA?5?$AAf?$AAo?$AAr?$AA?5?$AA_?$AAo@ 10001810     LIBCMT:crt0msg.obj
 0001:00000880       ??_C@_1FC@ECHBIFBC@?$AAR?$AA6?$AA0?$AA1?$AA9?$AA?$AN?$AA?6?$AA?9?$AA?5?$AAu?$AAn?$AAa?$AAb?$AAl?$AAe?$AA?5?$AAt?$AAo?$AA?5?$AAo?$AAp?$AAe?$AAn?$AA?5?$AAc?$AAo?$AAn?$AAs?$AAo?$AAl?$AAe?$AA?5@ 10001880     LIBCMT:crt0msg.obj
 0001:000008d8       ??_C@_1EC@JIBHAOPH@?$AAR?$AA6?$AA0?$AA1?$AA8?$AA?$AN?$AA?6?$AA?9?$AA?5?$AAu?$AAn?$AAe?$AAx?$AAp?$AAe?$AAc?$AAt?$AAe?$AAd?$AA?5?$AAh?$AAe?$AAa?$AAp?$AA?5?$AAe?$AAr?$AAr?$AAo?$AAr?$AA?$AN?$AA?6@ 100018d8     LIBCMT:crt0msg.obj
 0001:00000920       ??_C@_1FK@BEOGODMC@?$AAR?$AA6?$AA0?$AA1?$AA7?$AA?$AN?$AA?6?$AA?9?$AA?5?$AAu?$AAn?$AAe?$AAx?$AAp?$AAe?$AAc?$AAt?$AAe?$AAd?$AA?5?$AAm?$AAu?$AAl?$AAt?$AAi?$AAt?$AAh?$AAr?$AAe?$AAa?$AAd?$AA?5@ 10001920     LIBCMT:crt0msg.obj
 0001:00000980       ??_C@_1FI@LOGNIKDM@?$AAR?$AA6?$AA0?$AA1?$AA6?$AA?$AN?$AA?6?$AA?9?$AA?5?$AAn?$AAo?$AAt?$AA?5?$AAe?$AAn?$AAo?$AAu?$AAg?$AAh?$AA?5?$AAs?$AAp?$AAa?$AAc?$AAe?$AA?5?$AAf?$AAo?$AAr?$AA?5?$AAt?$AAh@ 10001980     LIBCMT:crt0msg.obj
 0001:000009d8       ??_C@_1EG@BEHAGFJD@?$AAR?$AA6?$AA0?$AA1?$AA0?$AA?$AN?$AA?6?$AA?9?$AA?5?$AAa?$AAb?$AAo?$AAr?$AAt?$AA?$CI?$AA?$CJ?$AA?5?$AAh?$AAa?$AAs?$AA?5?$AAb?$AAe?$AAe?$AAn?$AA?5?$AAc?$AAa?$AAl?$AAl?$AAe?$AAd@ 100019d8     LIBCMT:crt0msg.obj
 0001:00000a20       ??_C@_1FI@HONFMGBI@?$AAR?$AA6?$AA0?$AA0?$AA9?$AA?$AN?$AA?6?$AA?9?$AA?5?$AAn?$AAo?$AAt?$AA?5?$AAe?$AAn?$AAo?$AAu?$AAg?$AAh?$AA?5?$AAs?$AAp?$AAa?$AAc?$AAe?$AA?5?$AAf?$AAo?$AAr?$AA?5?$AAe?$AAn@ 10001a20     LIBCMT:crt0msg.obj
 0001:00000a78       ??_C@_1FE@LLNEDJMD@?$AAR?$AA6?$AA0?$AA0?$AA8?$AA?$AN?$AA?6?$AA?9?$AA?5?$AAn?$AAo?$AAt?$AA?5?$AAe?$AAn?$AAo?$AAu?$AAg?$AAh?$AA?5?$AAs?$AAp?$AAa?$AAc?$AAe?$AA?5?$AAf?$AAo?$AAr?$AA?5?$AAa?$AAr@ 10001a78     LIBCMT:crt0msg.obj
 0001:00000ad0       ??_C@_1FK@PGACCAFB@?$AAR?$AA6?$AA0?$AA0?$AA2?$AA?$AN?$AA?6?$AA?9?$AA?5?$AAf?$AAl?$AAo?$AAa?$AAt?$AAi?$AAn?$AAg?$AA?5?$AAp?$AAo?$AAi?$AAn?$AAt?$AA?5?$AAs?$AAu?$AAp?$AAp?$AAo?$AAr?$AAt?$AA?5@ 10001ad0     LIBCMT:crt0msg.obj
 0001:00000be0       ??_C@_1EK@MBDPDCGA@?$AAM?$AAi?$AAc?$AAr?$AAo?$AAs?$AAo?$AAf?$AAt?$AA?5?$AAV?$AAi?$AAs?$AAu?$AAa?$AAl?$AA?5?$AAC?$AA?$CL?$AA?$CL?$AA?5?$AAR?$AAu?$AAn?$AAt?$AAi?$AAm?$AAe?$AA?5?$AAL?$AAi?$AAb@ 10001be0     LIBCMT:crt0msg.obj
 0001:00000c2c       ??_C@_15IABLJNFO@?$AA?6?$AA?6?$AA?$AA@ 10001c2c     LIBCMT:crt0msg.obj
 0001:00000c34       ??_C@_17LGKOMLJ@?$AA?4?$AA?4?$AA?4?$AA?$AA@ 10001c34     LIBCMT:crt0msg.obj
 0001:00000c3c       ??_C@_1CO@EAEJAADC@?$AA?$DM?$AAp?$AAr?$AAo?$AAg?$AAr?$AAa?$AAm?$AA?5?$AAn?$AAa?$AAm?$AAe?$AA?5?$AAu?$AAn?$AAk?$AAn?$AAo?$AAw?$AAn?$AA?$DO?$AA?$AA@ 10001c3c     LIBCMT:crt0msg.obj
 0001:00000c6c       ??_C@_1DE@JNGNBFGO@?$AAR?$AAu?$AAn?$AAt?$AAi?$AAm?$AAe?$AA?5?$AAE?$AAr?$AAr?$AAo?$AAr?$AA?$CB?$AA?6?$AA?6?$AAP?$AAr?$AAo?$AAg?$AAr?$AAa?$AAm?$AA?3?$AA?5?$AA?$AA@ 10001c6c     LIBCMT:crt0msg.obj
 0001:00000ca0       ??_C@_1BK@DBDEIDLH@?$AAK?$AAE?$AAR?$AAN?$AAE?$AAL?$AA3?$AA2?$AA?4?$AAD?$AAL?$AAL?$AA?$AA@ 10001ca0     LIBCMT:tidtable.obj
 0001:00000cbc       ??_C@_07PEJMOBNF@FlsFree?$AA@ 10001cbc     LIBCMT:tidtable.obj
 0001:00000cc4       ??_C@_0M@JCPCPOEF@FlsSetValue?$AA@ 10001cc4     LIBCMT:tidtable.obj
 0001:00000cd0       ??_C@_0M@GDNOONDI@FlsGetValue?$AA@ 10001cd0     LIBCMT:tidtable.obj
 0001:00000cdc       ??_C@_08KNHFBNJ@FlsAlloc?$AA@ 10001cdc     LIBCMT:tidtable.obj
 0001:00000ce8       __XcptActTab               10001ce8     LIBCMT:winxfltr.obj
 0001:00000d78       __First_FPE_Indx           10001d78     LIBCMT:winxfltr.obj
 0001:00000d7c       __Num_FPE                  10001d7c     LIBCMT:winxfltr.obj
 0001:00000d80       __XcptActTabSize           10001d80     LIBCMT:winxfltr.obj
 0001:00000d84       __XcptActTabCount          10001d84     LIBCMT:winxfltr.obj
 0001:00000d88       ??_C@_0BI@DFKBFLJE@GetProcessWindowStation?$AA@ 10001d88     LIBCMT:crtmboxw.obj
 0001:00000da0       ??_C@_0BK@DEKFELLI@GetUserObjectInformationW?$AA@ 10001da0     LIBCMT:crtmboxw.obj
 0001:00000dbc       ??_C@_0BD@HHGDFDBJ@GetLastActivePopup?$AA@ 10001dbc     LIBCMT:crtmboxw.obj
 0001:00000dd0       ??_C@_0BA@HNOPNCHB@GetActiveWindow?$AA@ 10001dd0     LIBCMT:crtmboxw.obj
 0001:00000de0       ??_C@_0M@DLDCCGNP@MessageBoxW?$AA@ 10001de0     LIBCMT:crtmboxw.obj
 0001:00000dec       ??_C@_1BG@GOEBHBDC@?$AAU?$AAS?$AAE?$AAR?$AA3?$AA2?$AA?4?$AAD?$AAL?$AAL?$AA?$AA@ 10001dec     LIBCMT:crtmboxw.obj
 0001:00000e04       ??_C@_1BC@GDGBMEMK@?$AAH?$AAH?$AA?3?$AAm?$AAm?$AA?3?$AAs?$AAs?$AA?$AA@ 10001e04     LIBCMT:nlsdata2.obj
 0001:00000e18       ??_C@_1CI@KNAKOEBC@?$AAd?$AAd?$AAd?$AAd?$AA?0?$AA?5?$AAM?$AAM?$AAM?$AAM?$AA?5?$AAd?$AAd?$AA?0?$AA?5?$AAy?$AAy?$AAy?$AAy?$AA?$AA@ 10001e18     LIBCMT:nlsdata2.obj
 0001:00000e40       ??_C@_1BC@IEBCMHCM@?$AAM?$AAM?$AA?1?$AAd?$AAd?$AA?1?$AAy?$AAy?$AA?$AA@ 10001e40     LIBCMT:nlsdata2.obj
 0001:00000e54       ??_C@_15CLMNNGEL@?$AAP?$AAM?$AA?$AA@ 10001e54     LIBCMT:nlsdata2.obj
 0001:00000e5c       ??_C@_15ODEHAHHF@?$AAA?$AAM?$AA?$AA@ 10001e5c     LIBCMT:nlsdata2.obj
 0001:00000e64       ??_C@_1BC@FEMKIFH@?$AAD?$AAe?$AAc?$AAe?$AAm?$AAb?$AAe?$AAr?$AA?$AA@ 10001e64     LIBCMT:nlsdata2.obj
 0001:00000e78       ??_C@_1BC@BGLIFPF@?$AAN?$AAo?$AAv?$AAe?$AAm?$AAb?$AAe?$AAr?$AA?$AA@ 10001e78     LIBCMT:nlsdata2.obj
 0001:00000e8c       ??_C@_1BA@EPANDLNG@?$AAO?$AAc?$AAt?$AAo?$AAb?$AAe?$AAr?$AA?$AA@ 10001e8c     LIBCMT:nlsdata2.obj
 0001:00000e9c       ??_C@_1BE@DKAAMBJL@?$AAS?$AAe?$AAp?$AAt?$AAe?$AAm?$AAb?$AAe?$AAr?$AA?$AA@ 10001e9c     LIBCMT:nlsdata2.obj
 0001:00000eb0       ??_C@_1O@PAHLKOAC@?$AAA?$AAu?$AAg?$AAu?$AAs?$AAt?$AA?$AA@ 10001eb0     LIBCMT:nlsdata2.obj
 0001:00000ec0       ??_C@_19BIFMLPCD@?$AAJ?$AAu?$AAl?$AAy?$AA?$AA@ 10001ec0     LIBCMT:nlsdata2.obj
 0001:00000ecc       ??_C@_19EPFLPGAP@?$AAJ?$AAu?$AAn?$AAe?$AA?$AA@ 10001ecc     LIBCMT:nlsdata2.obj
 0001:00000ed8       ??_C@_1M@GJNLMHFD@?$AAA?$AAp?$AAr?$AAi?$AAl?$AA?$AA@ 10001ed8     LIBCMT:nlsdata2.obj
 0001:00000ee4       ??_C@_1M@IKEENEDF@?$AAM?$AAa?$AAr?$AAc?$AAh?$AA?$AA@ 10001ee4     LIBCMT:nlsdata2.obj
 0001:00000ef0       ??_C@_1BC@JGDDFFAM@?$AAF?$AAe?$AAb?$AAr?$AAu?$AAa?$AAr?$AAy?$AA?$AA@ 10001ef0     LIBCMT:nlsdata2.obj
 0001:00000f04       ??_C@_1BA@EFMEIEBA@?$AAJ?$AAa?$AAn?$AAu?$AAa?$AAr?$AAy?$AA?$AA@ 10001f04     LIBCMT:nlsdata2.obj
 0001:00000f14       ??_C@_17EGKACKIF@?$AAD?$AAe?$AAc?$AA?$AA@ 10001f14     LIBCMT:nlsdata2.obj
 0001:00000f1c       ??_C@_17BBDMLCIG@?$AAN?$AAo?$AAv?$AA?$AA@ 10001f1c     LIBCMT:nlsdata2.obj
 0001:00000f24       ??_C@_17FNLKOI@?$AAO?$AAc?$AAt?$AA?$AA@ 10001f24     LIBCMT:nlsdata2.obj
 0001:00000f2c       ??_C@_17HCHCOKMG@?$AAS?$AAe?$AAp?$AA?$AA@ 10001f2c     LIBCMT:nlsdata2.obj
 0001:00000f34       ??_C@_17ICPELBCN@?$AAA?$AAu?$AAg?$AA?$AA@ 10001f34     LIBCMT:nlsdata2.obj
 0001:00000f3c       ??_C@_17IJPCKHK@?$AAJ?$AAu?$AAl?$AA?$AA@ 10001f3c     LIBCMT:nlsdata2.obj
 0001:00000f44       ??_C@_17KCJGOCPB@?$AAJ?$AAu?$AAn?$AA?$AA@ 10001f44     LIBCMT:nlsdata2.obj
 0001:00000f4c       ??_C@_17PNNKMEED@?$AAM?$AAa?$AAy?$AA?$AA@ 10001f4c     LIBCMT:nlsdata2.obj
 0001:00000f54       ??_C@_17LFPOIHDD@?$AAA?$AAp?$AAr?$AA?$AA@ 10001f54     LIBCMT:nlsdata2.obj
 0001:00000f5c       ??_C@_17CKNLEDEC@?$AAM?$AAa?$AAr?$AA?$AA@ 10001f5c     LIBCMT:nlsdata2.obj
 0001:00000f64       ??_C@_17LMDJEKJN@?$AAF?$AAe?$AAb?$AA?$AA@ 10001f64     LIBCMT:nlsdata2.obj
 0001:00000f6c       ??_C@_17DKNBKCHM@?$AAJ?$AAa?$AAn?$AA?$AA@ 10001f6c     LIBCMT:nlsdata2.obj
 0001:00000f74       ??_C@_1BC@ENMNNPAJ@?$AAS?$AAa?$AAt?$AAu?$AAr?$AAd?$AAa?$AAy?$AA?$AA@ 10001f74     LIBCMT:nlsdata2.obj
 0001:00000f88       ??_C@_1O@PDICJHAG@?$AAF?$AAr?$AAi?$AAd?$AAa?$AAy?$AA?$AA@ 10001f88     LIBCMT:nlsdata2.obj
 0001:00000f98       ??_C@_1BC@HHMNLIHE@?$AAT?$AAh?$AAu?$AAr?$AAs?$AAd?$AAa?$AAy?$AA?$AA@ 10001f98     LIBCMT:nlsdata2.obj
 0001:00000fac       ??_C@_1BE@EBOGMDOH@?$AAW?$AAe?$AAd?$AAn?$AAe?$AAs?$AAd?$AAa?$AAy?$AA?$AA@ 10001fac     LIBCMT:nlsdata2.obj
 0001:00000fc0       ??_C@_1BA@ENFBFFEK@?$AAT?$AAu?$AAe?$AAs?$AAd?$AAa?$AAy?$AA?$AA@ 10001fc0     LIBCMT:nlsdata2.obj
 0001:00000fd0       ??_C@_1O@MMNBFLIA@?$AAM?$AAo?$AAn?$AAd?$AAa?$AAy?$AA?$AA@ 10001fd0     LIBCMT:nlsdata2.obj
 0001:00000fe0       ??_C@_1O@IHNHDHPB@?$AAS?$AAu?$AAn?$AAd?$AAa?$AAy?$AA?$AA@ 10001fe0     LIBCMT:nlsdata2.obj
 0001:00000ff0       ??_C@_17GGIBDPIH@?$AAS?$AAa?$AAt?$AA?$AA@ 10001ff0     LIBCMT:nlsdata2.obj
 0001:00000ff8       ??_C@_17HFOLPPLP@?$AAF?$AAr?$AAi?$AA?$AA@ 10001ff8     LIBCMT:nlsdata2.obj
 0001:00001000       ??_C@_17PDPHAADD@?$AAT?$AAh?$AAu?$AA?$AA@ 10002000     LIBCMT:nlsdata2.obj
 0001:00001008       ??_C@_17CJEDCEPE@?$AAW?$AAe?$AAd?$AA?$AA@ 10002008     LIBCMT:nlsdata2.obj
 0001:00001010       ??_C@_17BMKGEGOJ@?$AAT?$AAu?$AAe?$AA?$AA@ 10002010     LIBCMT:nlsdata2.obj
 0001:00001018       ??_C@_17KBOMKBF@?$AAM?$AAo?$AAn?$AA?$AA@ 10002018     LIBCMT:nlsdata2.obj
 0001:00001020       ??_C@_17MBGCMIPB@?$AAS?$AAu?$AAn?$AA?$AA@ 10002020     LIBCMT:nlsdata2.obj
 0001:00001028       ??_C@_08JCCMCCIL@HH?3mm?3ss?$AA@ 10002028     LIBCMT:nlsdata2.obj
 0001:00001034       ??_C@_0BE@CKGJFCPC@dddd?0?5MMMM?5dd?0?5yyyy?$AA@ 10002034     LIBCMT:nlsdata2.obj
 0001:00001048       ??_C@_08BPBNCDIB@MM?1dd?1yy?$AA@ 10002048     LIBCMT:nlsdata2.obj
 0001:00001054       ??_C@_02CJNFDJBF@PM?$AA@   10002054     LIBCMT:nlsdata2.obj
 0001:00001058       ??_C@_02DEDBPAFC@AM?$AA@   10002058     LIBCMT:nlsdata2.obj
 0001:0000105c       ??_C@_08EDHMEBNP@December?$AA@ 1000205c     LIBCMT:nlsdata2.obj
 0001:00001068       ??_C@_08HCHEGEOA@November?$AA@ 10002068     LIBCMT:nlsdata2.obj
 0001:00001074       ??_C@_07JJNFCEND@October?$AA@ 10002074     LIBCMT:nlsdata2.obj
 0001:0000107c       ??_C@_09BHHEALKD@September?$AA@ 1000207c     LIBCMT:nlsdata2.obj
 0001:00001088       ??_C@_06LBBHFDDG@August?$AA@ 10002088     LIBCMT:nlsdata2.obj
 0001:00001090       ??_C@_04MIEPOIFP@July?$AA@ 10002090     LIBCMT:nlsdata2.obj
 0001:00001098       ??_C@_04CNLMGBGM@June?$AA@ 10002098     LIBCMT:nlsdata2.obj
 0001:000010a0       ??_C@_05DMJDNLEJ@April?$AA@ 100020a0     LIBCMT:nlsdata2.obj
 0001:000010a8       ??_C@_05HPCKOFNC@March?$AA@ 100020a8     LIBCMT:nlsdata2.obj
 0001:000010b0       ??_C@_08GNJGEPFN@February?$AA@ 100020b0     LIBCMT:nlsdata2.obj
 0001:000010bc       ??_C@_07CGJPFGJA@January?$AA@ 100020bc     LIBCMT:nlsdata2.obj
 0001:000010c4       ??_C@_03MKABNOCG@Dec?$AA@  100020c4     LIBCMT:nlsdata2.obj
 0001:000010c8       ??_C@_03JPJOFNIA@Nov?$AA@  100020c8     LIBCMT:nlsdata2.obj
 0001:000010cc       ??_C@_03BMAOKBAD@Oct?$AA@  100020cc     LIBCMT:nlsdata2.obj
 0001:000010d0       ??_C@_03GGCAPAJC@Sep?$AA@  100020d0     LIBCMT:nlsdata2.obj
 0001:000010d4       ??_C@_03IFJFEIGA@Aug?$AA@  100020d4     LIBCMT:nlsdata2.obj
 0001:000010d8       ??_C@_03LBGABGKK@Jul?$AA@  100020d8     LIBCMT:nlsdata2.obj
 0001:000010dc       ??_C@_03IDFGHECI@Jun?$AA@  100020dc     LIBCMT:nlsdata2.obj
 0001:000010e0       ??_C@_03CNMDKL@May?$AA@    100020e0     LIBCMT:nlsdata2.obj
 0001:000010e4       ??_C@_03LEOLGMJP@Apr?$AA@  100020e4     LIBCMT:nlsdata2.obj
 0001:000010e8       ??_C@_03ODNJBKGA@Mar?$AA@  100020e8     LIBCMT:nlsdata2.obj
 0001:000010ec       ??_C@_03HJBDCHOM@Feb?$AA@  100020ec     LIBCMT:nlsdata2.obj
 0001:000010f0       ??_C@_03JIHJHPIE@Jan?$AA@  100020f0     LIBCMT:nlsdata2.obj
 0001:000010f4       ??_C@_08INBOOONO@Saturday?$AA@ 100020f4     LIBCMT:nlsdata2.obj
 0001:00001100       ??_C@_06JECMNKMI@Friday?$AA@ 10002100     LIBCMT:nlsdata2.obj
 0001:00001108       ??_C@_08HACCIKIA@Thursday?$AA@ 10002108     LIBCMT:nlsdata2.obj
 0001:00001114       ??_C@_09DLIGFAKA@Wednesday?$AA@ 10002114     LIBCMT:nlsdata2.obj
 0001:00001120       ??_C@_07BAAGCFCM@Tuesday?$AA@ 10002120     LIBCMT:nlsdata2.obj
 0001:00001128       ??_C@_06JLEDEDGH@Monday?$AA@ 10002128     LIBCMT:nlsdata2.obj
 0001:00001130       ??_C@_06OOPIFAJ@Sunday?$AA@ 10002130     LIBCMT:nlsdata2.obj
 0001:00001138       ??_C@_03FEFJNEK@Sat?$AA@   10002138     LIBCMT:nlsdata2.obj
 0001:0000113c       ??_C@_03IDIOELNC@Fri?$AA@  1000213c     LIBCMT:nlsdata2.obj
 0001:00001140       ??_C@_03IOFIKPDN@Thu?$AA@  10002140     LIBCMT:nlsdata2.obj
 0001:00001144       ??_C@_03MHOMLAJA@Wed?$AA@  10002144     LIBCMT:nlsdata2.obj
 0001:00001148       ??_C@_03NAGEINEP@Tue?$AA@  10002148     LIBCMT:nlsdata2.obj
 0001:0000114c       ??_C@_03PDAGKDH@Mon?$AA@   1000214c     LIBCMT:nlsdata2.obj
 0001:00001150       ??_C@_03KOEHGMDN@Sun?$AA@  10002150     LIBCMT:nlsdata2.obj
 0001:00001160       ___newctype                10002160     LIBCMT:ctype.obj
 0001:00001460       __wctype                   10002460     LIBCMT:ctype.obj
 0001:00001668       ___newclmap                10002668     LIBCMT:ctype.obj
 0001:000017e8       ___newcumap                100027e8     LIBCMT:ctype.obj
 0001:00001968       __load_config_used         10002968     LIBCMT:loadcfg.obj
 0001:000019b0       ___safe_se_handler_table   100029b0     <linker-defined>
 0001:000019bc       ___rtc_iaa                 100029bc     LIBCMT:_initsect_.obj
 0001:000019c0       ___rtc_izz                 100029c0     LIBCMT:_initsect_.obj
 0001:000019c4       ___rtc_taa                 100029c4     LIBCMT:_initsect_.obj
 0001:000019c8       ___rtc_tzz                 100029c8     LIBCMT:_initsect_.obj
 0001:000019d0       __alloca_probe             100029d0     chkstk.obj
 0001:000019d0       __chkstk                   100029d0 f   chkstk.obj
 0001:00001a00       _GetGlobalInfoW@4          10002a00 f   EditCase.obj
 0001:00001a80       _SetStartupInfoW@4         10002a80 f   EditCase.obj
 0001:00001c60       _ExitFARW@4                10002c60 f   EditCase.obj
 0001:00001c70       ?FindStart@@YAHPA_WHH@Z    10002c70 f   EditCase.obj
 0001:00001cc0       ?FindEnd@@YAHPA_WHH@Z      10002cc0 f   EditCase.obj
 0001:00001d10       ?ChangeCase@@YAHPA_WHHH@Z  10002d10 f   EditCase.obj
 0001:00001e00       _GetPluginInfoW@4          10002e00 f   EditCase.obj
 0001:00001e50       ?FindBounds@@YA_NPA_WHHAAH1@Z 10002e50 f   EditCase.obj
 0001:00002080       ?GetNextCCType@@YAHPA_WHHH@Z 10003080 f   EditCase.obj
 0001:00002210       _OpenW@4                   10003210 f   EditCase.obj
 0001:00002620       _memcpy                    10003620 f   LIBCMT:memcpy.obj
 0001:00002981       _malloc                    10003981 f   LIBCMT:malloc.obj
 0001:00002a15       _free                      10003a15 f   LIBCMT:free.obj
 0001:00002a50       _memset                    10003a50 f   LIBCMT:memset.obj
 0001:00002ad0       __ftol2_sse                10003ad0 f   LIBCMT:ftol2.obj
 0001:00002ad9       __ftol2_pentium4           10003ad9 f   LIBCMT:ftol2.obj
 0001:00002aec       __ftol2_sse_excpt          10003aec f   LIBCMT:ftol2.obj
 0001:00002b06       __ftol2                    10003b06 f   LIBCMT:ftol2.obj
 0001:00002b7b       __CRT_INIT@12              10003b7b f   LIBCMT:dllcrt0.obj
 0001:00002dd5       __DllMainCRTStartup@12     10003dd5 f   LIBCMT:dllcrt0.obj
 0001:00002df8       __VEC_memcpy               10003df8 f   LIBCMT:p4_memcpy.obj
 0001:00002efb       ___sse2_available_init     10003efb f   LIBCMT:cpu_disp.obj
 0001:00002f0b       ___crtCorExitProcess       10003f0b f   LIBCMT:crt0dat.obj
 0001:00002f36       ___crtExitProcess          10003f36 f   LIBCMT:crt0dat.obj
 0001:00002f4e       __lockexit                 10003f4e f   LIBCMT:crt0dat.obj
 0001:00002f57       __unlockexit               10003f57 f   LIBCMT:crt0dat.obj
 0001:00002f60       __init_pointers            10003f60 f   LIBCMT:crt0dat.obj
 0001:00002f93       __initterm_e               10003f93 f   LIBCMT:crt0dat.obj
 0001:00002fb7       __cinit                    10003fb7 f   LIBCMT:crt0dat.obj
 0001:0000318e       __exit                     1000418e f   LIBCMT:crt0dat.obj
 0001:000031a4       __cexit                    100041a4 f   LIBCMT:crt0dat.obj
 0001:000031b3       __amsg_exit                100041b3 f   LIBCMT:crt0dat.obj
 0001:000031d1       __GET_RTERRMSG             100041d1 f   LIBCMT:crt0msg.obj
 0001:000031f7       __NMSG_WRITE               100041f7 f   LIBCMT:crt0msg.obj
 0001:000033a6       __FF_MSGBANNER             100043a6 f   LIBCMT:crt0msg.obj
 0001:000033df       __heap_init                100043df f   LIBCMT:heapinit.obj
 0001:000033fd       __heap_term                100043fd f   LIBCMT:heapinit.obj
 0001:00003411       __get_errno_from_oserr     10004411 f   LIBCMT:dosmap.obj
 0001:00003453       __errno                    10004453 f   LIBCMT:dosmap.obj
 0001:00003466       __initp_heap_handler       10004466 f   LIBCMT:handler.obj
 0001:00003475       __callnewh                 10004475 f   LIBCMT:handler.obj
 0001:0000349d       __VEC_memzero              1000449d f   LIBCMT:p4_memset.obj
 0001:00003557       __encoded_null             10004557 f   LIBCMT:tidtable.obj
 0001:00003560       ___crtTlsAlloc@4           10004560 f   LIBCMT:tidtable.obj
 0001:00003569       ___set_flsgetvalue         10004569 f   LIBCMT:tidtable.obj
 0001:0000359d       __mtterm                   1000459d f   LIBCMT:tidtable.obj
 0001:000035da       __initptd                  100045da f   LIBCMT:tidtable.obj
 0001:0000368e       __getptd_noexit            1000468e f   LIBCMT:tidtable.obj
 0001:00003707       __getptd                   10004707 f   LIBCMT:tidtable.obj
 0001:00003721       __freefls@4                10004721 f   LIBCMT:tidtable.obj
 0001:00003850       __freeptd                  10004850 f   LIBCMT:tidtable.obj
 0001:000038be       __mtinit                   100048be f   LIBCMT:tidtable.obj
 0001:00003a39       __malloc_crt               10004a39 f   LIBCMT:crtheap.obj
 0001:00003a7e       __calloc_crt               10004a7e f   LIBCMT:crtheap.obj
 0001:00003aca       __realloc_crt              10004aca f   LIBCMT:crtheap.obj
 0001:00003b18       __ioinit                   10004b18 f   LIBCMT:ioinit.obj
 0001:00003d5d       __ioterm                   10004d5d f   LIBCMT:ioinit.obj
 0001:00003db0       __setenvp                  10004db0 f   LIBCMT:stdenvp.obj
 0001:00004026       __setargv                  10005026 f   LIBCMT:stdargv.obj
 0001:000040e1       ___crtGetEnvironmentStringsA 100050e1 f   LIBCMT:a_env.obj
 0001:00004178       __RTC_Initialize           10005178 f   LIBCMT:_initsect_.obj
 0001:0000419e       __RTC_Terminate            1000519e f   LIBCMT:_initsect_.obj
 0001:000041d0       __SEH_prolog4              100051d0 f   LIBCMT:sehprolg4.obj
 0001:00004215       __SEH_epilog4              10005215 f   LIBCMT:sehprolg4.obj
 0001:00004230       __except_handler4          10005230 f   LIBCMT:chandler4.obj
 0001:000043bf       __XcptFilter               100053bf f   LIBCMT:winxfltr.obj
 0001:00004509       ___CppXcptFilter           10005509 f   LIBCMT:winxfltr.obj
 0001:00004529       _DllMain@12                10005529 f   LIBCMT:dllmain.obj
 0001:0000452f       ___security_init_cookie    1000552f f   LIBCMT:gs_support.obj
 0001:000045ca       __mtinitlocks              100055ca f   LIBCMT:mlock.obj
 0001:00004614       __mtdeletelocks            10005614 f   LIBCMT:mlock.obj
 0001:0000466b       __unlock                   1000566b f   LIBCMT:mlock.obj
 0001:00004682       __mtinitlocknum            10005682 f   LIBCMT:mlock.obj
 0001:00004744       __lock                     10005744 f   LIBCMT:mlock.obj
 0001:00004777       ?terminate@@YAXXZ          10005777 f   LIBCMT:hooks.obj
 0001:000047b0       __initp_eh_hooks           100057b0 f   LIBCMT:hooks.obj
 0001:000047c1       __initp_misc_winsig        100057c1 f   LIBCMT:winsig.obj
 0001:00004816       ___get_sigabrt             10005816 f   LIBCMT:winsig.obj
 0001:00004823       _raise                     10005823 f   LIBCMT:winsig.obj
 0001:000049c6       __initp_misc_rand_s        100059c6 f   LIBCMT:rand_s.obj
 0001:000049d5       __initp_misc_purevirt      100059d5 f   LIBCMT:inithelp.obj
 0001:000049e4       __initp_misc_invarg        100059e4 f   LIBCMT:invarg.obj
 0001:000049f3       __call_reportfault         100059f3 f   LIBCMT:invarg.obj
 0001:00004b1c       __invoke_watson            10005b1c f   LIBCMT:invarg.obj
 0001:00004b41       __invalid_parameter        10005b41 f   LIBCMT:invarg.obj
 0001:00004b6e       __invalid_parameter_noinfo 10005b6e f   LIBCMT:invarg.obj
 0001:00004c34       ___onexitinit              10005c34 f   LIBCMT:onexit.obj
 0001:00004c65       __onexit                   10005c65 f   LIBCMT:onexit.obj
 0001:00004ca1       _atexit                    10005ca1 f   LIBCMT:onexit.obj
 0001:00004cb8       __initp_misc_cfltcvt_tab   10005cb8 f   LIBCMT:cmiscdat.obj
 0001:00004ce0       __ValidateImageBase        10005ce0 f   LIBCMT:pesect.obj
 0001:00004d20       __FindPESection            10005d20 f   LIBCMT:pesect.obj
 0001:00004d70       __IsNonwritableInCurrentImage 10005d70 f   LIBCMT:pesect.obj
 0001:00004e30       _strlen                    10005e30 f   LIBCMT:strlen.obj
 0001:00004ebb       ___crtMessageBoxW          10005ebb f   LIBCMT:crtmboxw.obj
 0001:00005027       _wcscat_s                  10006027 f   LIBCMT:wcscat_s.obj
 0001:0000509c       _wcsncpy_s                 1000609c f   LIBCMT:wcsncpy_s.obj
 0001:00005169       _wcslen                    10006169 f   LIBCMT:wcslen.obj
 0001:00005184       _wcscpy_s                  10006184 f   LIBCMT:wcscpy_s.obj
 0001:000051e7       __set_error_mode           100061e7 f   LIBCMT:errmode.obj
 0001:00005226       @__security_check_cookie@4 10006226 f   LIBCMT:secchk.obj
 0001:00005235       ___addlocaleref            10006235 f   LIBCMT:localref.obj
 0001:000052c4       ___removelocaleref         100062c4 f   LIBCMT:localref.obj
 0001:0000535d       ___freetlocinfo            1000635d f   LIBCMT:localref.obj
 0001:000054a8       __updatetlocinfoEx_nolock  100064a8 f   LIBCMT:localref.obj
 0001:000054f5       ___updatetlocinfo          100064f5 f   LIBCMT:localref.obj
 0001:00005791       ___updatetmbcinfo          10006791 f   LIBCMT:mbctype.obj
 0001:00005835       ??0_LocaleUpdate@@QAE@PAUlocaleinfo_struct@@@Z 10006835 f i LIBCMT:mbctype.obj
 0001:00005938       __setmbcp_nolock           10006938 f   LIBCMT:mbctype.obj
 0001:00005b21       __setmbcp                  10006b21 f   LIBCMT:mbctype.obj
 0001:00005cbb       ___initmbctable            10006cbb f   LIBCMT:mbctype.obj
 0001:00005cd9       __calloc_impl              10006cd9 f   LIBCMT:calloc_impl.obj
 0001:00005d5b       _realloc                   10006d5b f   LIBCMT:realloc.obj
 0001:00005e08       _strcpy_s                  10006e08 f   LIBCMT:strcpy_s.obj
 0001:00005eba       __ismbblead                10006eba f   LIBCMT:ismbbyte.obj
 0001:00005ee0       __local_unwind4            10006ee0 f   LIBCMT:exsup4.obj
 0001:00005fb6       __seh_longjmp_unwind4@4    10006fb6 f   LIBCMT:exsup4.obj
 0001:00005fd2       @_EH4_CallFilterFunc@8     10006fd2 f   LIBCMT:exsup4.obj
 0001:00005fe9       @_EH4_TransferToHandler@8  10006fe9 f   LIBCMT:exsup4.obj
 0001:00006002       @_EH4_GlobalUnwind2@8      10007002 f   LIBCMT:exsup4.obj
 0001:0000601b       @_EH4_LocalUnwind@16       1000701b f   LIBCMT:exsup4.obj
 0001:00006032       _abort                     10007032 f   LIBCMT:abort.obj
 0001:00006065       __freea                    10007065 f i LIBCMT:a_loc.obj
 0001:00006085       __crt_debugger_hook        10007085 f   LIBCMT:dbghook.obj
 0001:0000608d       __msize                    1000708d f   LIBCMT:msize.obj
 0001:000060c0       __fptrap                   100070c0 f   LIBCMT:crt0fp.obj
 0001:000060c9       ___report_gsfailure        100070c9 f   LIBCMT:gs_report.obj
 0001:000061cf       ___free_lc_time            100071cf f   LIBCMT:inittime.obj
 0001:00006546       ___free_lconv_num          10007546 f   LIBCMT:initnum.obj
 0001:000065af       ___free_lconv_mon          100075af f   LIBCMT:initmon.obj
 0001:00006894       ___crtLCMapStringA         10007894 f   LIBCMT:a_map.obj
 0001:000069c1       ___crtGetStringTypeA       100079c1 f   LIBCMT:a_str.obj
 0001:00006a10       __global_unwind2           10007a10 f   LIBCMT:exsup.obj
 0001:00006a75       __local_unwind2            10007a75 f   LIBCMT:exsup.obj
 0001:00006af9       __abnormal_termination     10007af9 f   LIBCMT:exsup.obj
 0001:00006b1c       __NLG_Notify1              10007b1c f   LIBCMT:exsup.obj
 0001:00006b25       __NLG_Notify               10007b25 f   LIBCMT:exsup.obj
 0001:00006b3c       __NLG_Dispatch2            10007b3c     LIBCMT:exsup.obj
 0001:00006b3c       __NLG_Dispatch             10007b3c     LIBCMT:exsup.obj
 0001:00006b44       __NLG_Call                 10007b44 f   LIBCMT:exsup.obj
 0001:00006b46       __NLG_Return2              10007b46     LIBCMT:exsup.obj
 0001:00006b50       __alloca_probe_16          10007b50 f   LIBCMT:alloca16.obj
 0001:00006b66       __alloca_probe_8           10007b66     LIBCMT:alloca16.obj
 0001:00006b7c       _RtlUnwind@16              10007b7c f   kernel32:KERNEL32.dll
 0001:00006d34       __IMPORT_DESCRIPTOR_KERNEL32 10007d34     kernel32:KERNEL32.dll
 0001:00006d48       __NULL_IMPORT_DESCRIPTOR   10007d48     kernel32:KERNEL32.dll
 0002:000001a0       ___flsindex                100091a0     LIBCMT:tidtable.obj
 0002:000001a4       ___getvalueindex           100091a4     LIBCMT:tidtable.obj
 0002:000001a8       ___badioinfo               100091a8     LIBCMT:ioinit.obj
 0002:00000310       __cfltcvt_tab              10009310     LIBCMT:cmiscdat.obj
 0002:00000340       ___security_cookie         10009340     LIBCMT:gs_cookie.obj
 0002:00000344       ___security_cookie_complement 10009344     LIBCMT:gs_cookie.obj
 0002:00000348       ___clocalestr              10009348     LIBCMT:nlsdata2.obj
 0002:00000350       ___lc_time_c               10009350     LIBCMT:nlsdata2.obj
 0002:000004b8       ___initiallocinfo          100094b8     LIBCMT:nlsdata2.obj
 0002:00000590       ___ptlocinfo               10009590     LIBCMT:nlsdata2.obj
 0002:00000598       ___initialmbcinfo          10009598     LIBCMT:mbctype.obj
 0002:000007b8       __mbctype                  100097b8     LIBCMT:mbctype.obj
 0002:000008c0       __mbcasemap                100098c0     LIBCMT:mbctype.obj
 0002:000009c0       ___ptmbcinfo               100099c0     LIBCMT:mbctype.obj
 0002:00000ac0       ___abort_behavior          10009ac0     LIBCMT:abort.obj
 0002:00000ac8       ___lconv_static_decimal    10009ac8     LIBCMT:lconv.obj
 0002:00000acc       ___lconv_static_W_decimal  10009acc     LIBCMT:lconv.obj
 0002:00000ad0       ___lconv_c                 10009ad0     LIBCMT:lconv.obj
 0002:00000b20       ___lconv                   10009b20     LIBCMT:lconv.obj
 0002:00000b24       ___globallocalestatus      10009b24     LIBCMT:glstatus.obj
 0002:00000b28       __pctype                   10009b28     LIBCMT:ctype.obj
 0002:00000b2c       __pwctype                  10009b2c     LIBCMT:ctype.obj
 0002:00000b30       __NLG_Destination          10009b30     LIBCMT:exsup.obj
 0002:00000c98       __aenvptr                  10009c98     LIBCMT:dllcrt0.obj
 0002:00000c9c       __wenvptr                  10009c9c     LIBCMT:dllcrt0.obj
 0002:00000ca0       ___error_mode              10009ca0     LIBCMT:dllcrt0.obj
 0002:00000ca4       ___app_type                10009ca4     LIBCMT:dllcrt0.obj
 0002:00000ca8       __umaskval                 10009ca8     LIBCMT:crt0dat.obj
 0002:00000cac       ___argc                    10009cac     LIBCMT:crt0dat.obj
 0002:00000cb0       ___argv                    10009cb0     LIBCMT:crt0dat.obj
 0002:00000cb4       ___wargv                   10009cb4     LIBCMT:crt0dat.obj
 0002:00000cb8       __environ                  10009cb8     LIBCMT:crt0dat.obj
 0002:00000cbc       ___initenv                 10009cbc     LIBCMT:crt0dat.obj
 0002:00000cc0       __wenviron                 10009cc0     LIBCMT:crt0dat.obj
 0002:00000cc4       ___winitenv                10009cc4     LIBCMT:crt0dat.obj
 0002:00000cc8       __pgmptr                   10009cc8     LIBCMT:crt0dat.obj
 0002:00000ccc       __wpgmptr                  10009ccc     LIBCMT:crt0dat.obj
 0002:00000cd0       __exitflag                 10009cd0     LIBCMT:crt0dat.obj
 0002:00000cd4       __C_Termination_Done       10009cd4     LIBCMT:crt0dat.obj
 0002:00000cd8       __C_Exit_Done              10009cd8     LIBCMT:crt0dat.obj
 0002:00001308       __crtheap                  1000a308     LIBCMT:heapinit.obj
 0002:0000130c       ?_pnhHeap@@3P6AHI@ZA       1000a30c     LIBCMT:handler.obj
 0002:00001310       __newmode                  1000a310     LIBCMT:_newmode.obj
 0002:00001314       _gpFlsAlloc                1000a314     LIBCMT:tidtable.obj
 0002:00001318       _gpFlsGetValue             1000a318     LIBCMT:tidtable.obj
 0002:0000131c       _gpFlsSetValue             1000a31c     LIBCMT:tidtable.obj
 0002:00001320       _gpFlsFree                 1000a320     LIBCMT:tidtable.obj
 0002:00001324       __maxwait                  1000a324     LIBCMT:crtheap.obj
 0002:00001580       ?__pInconsistency@@3P6AXXZA 1000a580     LIBCMT:hooks.obj
 0002:0000159c       ___pPurecall               1000a59c     LIBCMT:inithelp.obj
 0002:000015a0       ___pInvalidArgHandler      1000a5a0     LIBCMT:invarg.obj
 0002:000015bc       ___mbulinfo                1000a5bc     LIBCMT:mbctype.obj
 0002:000015c8       ___mbcodepage              1000a5c8     LIBCMT:mbctype.obj
 0002:000015cc       ___ismbcodepage            1000a5cc     LIBCMT:mbctype.obj
 0002:000015d0       ___mblcid                  1000a5d0     LIBCMT:mbctype.obj
 0002:000018fc       ___lconv_static_null       1000a8fc     LIBCMT:lconv.obj
 0002:00001900       ___lconv_static_W_null     1000a900     LIBCMT:lconv.obj
 0002:00001904       __debugger_hook_dummy      1000a904     <common>
 0002:00001908       __pDestructExceptionObject 1000a908     <common>
 0002:0000190c       __nhandle                  1000a90c     <common>
 0002:00001920       ___pioinfo                 1000a920     <common>
 0002:00001a20       ___env_initialized         1000aa20     <common>
 0002:00001a24       ___onexitend               1000aa24     <common>
 0002:00001a28       ___onexitbegin             1000aa28     <common>
 0002:00001a2c       ___mbctype_initialized     1000aa2c     <common>
 0002:00001a30       __FPinit                   1000aa30     <common>
 0002:00001a34       ___dyn_tls_init_callback   1000aa34     <common>
 0002:00001a38       ___sse2_available          1000aa38     <common>
 0002:00001a3c       __acmdln                   1000aa3c     <common>

 entry point at        0001:00002dd5

 Static symbols

 0001:00002cdf       ___DllMainCRTStartup       10003cdf f   LIBCMT:dllcrt0.obj
 0001:0000304e       _doexit                    1000404e f   LIBCMT:crt0dat.obj
 0001:00003e8c       _parse_cmdline             10004e8c f   LIBCMT:stdargv.obj
 0001:000047df       _siglookup                 100057df f   LIBCMT:winsig.obj
 0001:00004b7e       __onexit_nolock            10005b7e f   LIBCMT:onexit.obj
 0001:0000556e       ?CPtoLCID@@YAHH@Z          1000656e f   LIBCMT:mbctype.obj
 0001:0000559d       ?setSBCS@@YAXPAUthreadmbcinfostruct@@@Z 1000659d f   LIBCMT:mbctype.obj
 0001:00005601       ?setSBUpLow@@YAXPAUthreadmbcinfostruct@@@Z 10006601 f   LIBCMT:mbctype.obj
 0001:000058bc       ?getSystemCP@@YAHH@Z       100068bc f   LIBCMT:mbctype.obj
 0001:00005e67       ?x_ismbbtype_l@@YAHPAUlocaleinfo_struct@@IHH@Z 10006e67 f   LIBCMT:ismbbyte.obj
 0001:00005f70       __unwind_handler4          10006f70 f   LIBCMT:exsup4.obj
 0001:000066ad       ?__crtLCMapStringA_stat@@YAHPAUlocaleinfo_struct@@KKPBDHPADHHH@Z 100076ad f   LIBCMT:a_map.obj
 0001:000068da       ?__crtGetStringTypeA_stat@@YAHPAUlocaleinfo_struct@@KPBDHPAGHHH@Z 100078da f   LIBCMT:a_str.obj
 0001:00006a30       __unwind_handler           10007a30 f   LIBCMT:exsup.obj
